:020000020000FC
:1000000011C109C009C009C009C076C076C077C057
:10001000E8C007C173C0189518951895CF93DF9362
:100020001F922F921F931FB71F9365FB8EF563FBE3
:10003000BEF410B316FBA6F4109075001394109242
:10004000750013E0111661F4677FF0927300F0926F
:100050007400F09275001091A50012601093A50035
:10006000C0917300D0917400209769F419B71F7B79
:1000700019BF1091A5001E7F1093A5009498959824
:10008000C298C39831C02197C0937300D093740075
:1000900010906000212C1694279418F0C298C39AEF
:1000A00002C0C398C29A122C1694279418F0949800
:1000B000959A03C09598949A00C02092600011E030
:1000C0002090A700210E2092A7001091A6001F1DCE
:1000D0001093A6001AB510906100110E1BB5209068
:1000E0006200211E2BBC1ABC1F911FBF1F912F90B5
:1000F0001F90DF91CF9118951895189518952F930B
:100100003F930F92AF93BF93EF93FF931F922F9262
:100110003F921F931FB71F9323E61BB114FB76F981
:1001200010FB2EF01CB1312E77FB36F011C01CB144
:10013000312E1AB111FB66F010907200112009F4F3
:1001400042C010906E0020906F00121834F132C03F
:1001500010919F001F71232C269426942694211A17
:1001600031F0F0927200F0926E0078682CC07068E6
:10017000777F1AE0109376001FEF10937200F092D1
:100180006E0017E03122E3E6F1E08894EE1FFF1FD6
:10019000E30DFF1DC89500926F0030916E00230F94
:1001A000BB27A22F3C92339530936E001AE0109338
:1001B000760009C030916E00230FBB27A22F3C921E
:1001C0001FEF109371001F911FBF1F913F902F9041
:1001D0001F90FF91EF91BF91AF910F903F912F91A1
:1001E0001895AF93BF931F931FB71F931091700083
:1001F000139510937000155041F0A9E6109170000E
:10020000A10FBB271C911CB906C053985598F092BA
:100210006B00F0926C001F911FBF1F91BF91AF91B7
:10022000189518951FED1DBFFF24A0E6B0E0FD92C4
:1002300019ED1A1BE1F71FE015BF10E01BBF10E01E
:1002400019BF12E013BF10E01FBD13E41EBDA89537
:1002500018E011BD112718BB12BB1CEF17BB10E330
:1002600011BB14E91AB91CE019B913E018B92FD061
:10027000A9D1DFD102D27894DD24F2BE8CE792B707
:100280009817EAF31CE7810FE7E5F1E013E0D122CC
:10029000ED2C8894EE1C8894EE1FFF1FEE0DFF1DC1
:1002A000C895E7E5F1E0E00DFF1DD3940994040043
:1002B000060008000A0034D0E2CF85D1E0CFBAD1E1
:1002C000DECFDCD1DCCF0305020101010302772779
:1002D00066271DE210936000C298C3989498959881
:1002E00027E03327AEE9B0E01CB310FBEEF33EBBD2
:1002F00011E01CBB1DB31D9333952A952223A1F752
:1003000016B310FB70F90EF0529811FB2EF017E6A1
:1003100019B9F0929F00089510919E0019B908959F
:1003200010907100112009F413C1F0927100E8EAF5
:10033000F1E0109063008894111C8894EE1FFF1F59
:10034000E10DFF1DC895E8EAF1E0E00DFF1D0994FD
:100350000800420066008F009000AF00B000CE00A1
:100360006F7D1091A50015601093A500F092A60076
:10037000F092A70003D12091640024FB96F0109125
:10038000A5001B7F1093A5001091650010936200DB
:10039000109166001093610011E610937A00DAD094
:1003A000D6C01091650010937900109166001093EB
:1003B00078001091A300109362001091A400109394
:1003C00061001091A20010937B0011E010937A005D
:1003D000C1D0BDC01091640013FB63F9F0927500A9
:1003E000CDD0F092A600F092A70060621091A50017
:1003F00011601D7F1093A500109167001093740089
:1004000010916800109373001091650010936200C2
:1004100010916600109361009DD099C01091A500C5
:1004200014601093A50060611091A50010FB0EF000
:100430008EC0309164003093790020916500209344
:1004400078004091610050916200421B530B38F0DC
:10045000452B442339F011E010937A0003C012E0D9
:1004600010937A001091A20010937B0070C06FC0AF
:100470006B7E2091640021FB5EF41FEF10937800E7
:100480001093790012E010937A0020FB62F95FC0AC
:100490001091A5001E7F1093A50020FB26F09498D4
:1004A0009598C298C39819B71F7B19BF50C04FC009
:1004B0001091640010FB56F0A0EAB0E010916500C6
:1004C000A10FBF1D109166001C9341C01CB311FB0E
:1004D000EEF3109165001EBB109166001DBBF894F1
:1004E00014E01CBB12E01CBB789431C01091640076
:1004F00010FBFEF011FB66F0A0EAB0E01091650081
:10050000A10FBF1DF0926B001C9110936C001FC0D7
:10051000A0EAB0E010916500A10FBF1D1D912C91C4
:100520003E91311B3323A1F710936B0020936C0095
:100530000EC01CB310FBEEF3109165001EBB11E062
:100540001CBB2DB3F0926B0020936C0000C0746054
:10055000A895089519B71F7B19BF1CB510906100AD
:10056000110E1DB520906200211E2BBC1ABC18B7BD
:10057000106418BF19B7106419BF0895F8941EB518
:100580001C7F2091640023952370122B1EBD78944C
:100590002091640022FB66F910916000107C16F433
:1005A0002DE201C02EE1322F3695279527953FB7D2
:1005B000220F3FBF2795322F307C311BA1F72093AC
:1005C00060000895089577FB0EF031C0579872FBD4
:1005D0002EF4737710919F0010680DC02091760063
:1005E0002A952093760019F573FB77770EF41FC0D8
:1005F00010919F001F7776FB16F910936900F09217
:100600007200F0926E001091690020916A00120F42
:1006100020916B00120F20916C00120F10936D004F
:10062000F092700010916900539A1CB9559A579A2C
:100630000895089550907700552009F41DC0ACE34B
:10064000AB5350906400A51918F4F092770014C0D1
:10065000F0927700EBE3F3E0509064008894551C2F
:100660008894EE1FFF1FE50DFF1DC895EBE3F3E037
:10067000E00DFF1D099401000895089510917B007D
:10068000112321F01A9510937B0080C0A1E6AE558E
:1006900070907A00A71908F479C0EEE5F3E0709045
:1006A0007A008894771C8894EE1FFF1FE70DFF1DCA
:1006B000C895EEE5F3E0E00DFF1D0994030004008A
:1006C0002D0064C01091A20010937B002091610066
:1006D000309162004091A1005091A000241B350B85
:1006E00038F04091780050917900421B530B60F034
:1006F000209178003091790010E010937A001091E9
:10070000A5001B7F1093A500F894209361003093FF
:10071000620078943BC01091A20010937B0020915E
:100720006100309162004091A1005091A000240F1F
:10073000351F98F04091780050917900421B530B7F
:10074000F894209361003093620078942091A10086
:100750003091A000241B350BC8F064FB36F41091D7
:10076000A5001B7F1093A5000EC01091A5001E7F51
:100770001093A50019B71F7B19BF62FB26F0949850
:0E0780009598C298C39810E010937A000895DF
:00000001FF
